:100000000C9472000C948D000C948D000C948D0057
:100010000C948D000C948D000C948D000C948D002C
:100020000C948D000C948D000C948D000C948D001C
:100030000C948D000C948D000C948D000C948D000C
:100040000C948D000C948D000C948D000C948D00FC
:100050000C948D000C948D000C948D000C948D00EC
:100060000C948D000C948D000C948D000C948D00DC
:100070000C948D000C948D000C948D000C948D00CC
:100080000C948D000C948D000C948D000C948D00BC
:100090000C948D000C948D000C948D000C948D00AC
:1000A0000C948D000C948D000C948D000C948D009C
:1000B0000C948D000C948D000C948D000C948D008C
:1000C0000C948D000C948D000C948D000C948D007C
:1000D0000C948D000C948D000C948D000C948D006C
:1000E0000C948D0011241FBECFEFD1E2DEBFCDBF37
:1000F00000E00CBF84B78093000214BE0FB6F894E2
:10010000A8958091600088618093600010926000E3
:100110000FBE0E94AB000C94C6000C94000081B38B
:100120008F5F81BB8091080181508093080180918D
:100130000B01882371F080910B01880F80930B01D4
:100140008FE891E00197F1F700C0000090E080E0B7
:10015000089581E0F3CFF8948FEF80BB809307017F
:1001600080930A0111BA1092080110920B01789441
:1001700088E19EE00FB6F894A895809360000FBECA
:1001800090936000A8950E948F00FCCFF894FFCF59
:00000001FF
